:100000000C9462010C9474130C94A1130C948A0147
:100010000C948A010C948A010C948A010C948A0134
:100020000C948A010C948A010C948A010C948A0124
:100030000C948A010C948A010C948A010C948A0114
:100040000C9408170C948A010C94B5140C940715A1
:100050000C948A010C948A010C948A010C948A01F4
:100060000C948A010C948A01000021104220633014
:100070008440A550C660E770088129914AA16BB100
:100080008CC1ADD1CEE1EFF13112100273325222A8
:10009000B5529442F772D662399318837BB35AA350
:1000A000BDD39CC3FFF3DEE3622443342004011478
:1000B000E664C774A44485546AA54BB528850995A0
:1000C000EEE5CFF5ACC58DD5533672261116300648
:1000D000D776F6669556B4465BB77AA719973887F0
:1000E000DFF7FEE79DD7BCC7C448E5588668A77808
:1000F0004008611802282338CCC9EDD98EE9AFF940
:10010000488969990AA92BB9F55AD44AB77A966AE7
:10011000711A500A333A122AFDDBDCCBBFFB9EEB8F
:10012000799B588B3BBB1AABA66C877CE44CC55CB7
:10013000222C033C600C411CAEED8FFDECCDCDDDDF
:100140002AAD0BBD688D499D977EB66ED55EF44E87
:10015000133E322E511E700E9FFFBEEFDDDFFCCF2F
:100160001BBF3AAF599F788F8891A981CAB1EBA183
:100170000CD12DC14EF16FE18010A100C230E320FF
:100180000450254046706760B9839893FBA3DAB3A7
:100190003DC31CD37FE35EF3B1029012F322D2324F
:1001A0003542145277625672EAB5CBA5A895898577
:1001B0006EF54FE52CD50DC5E234C324A01481049F
:1001C0006674476424540544DBA7FAB79987B89747
:1001D0005FE77EF71DC73CD7D326F2369106B016EF
:1001E00057667676154634564CD96DC90EF92FE907
:1001F000C899E9898AB9ABA944586548067827683F
:10020000C018E1088238A3287DCB5CDB3FEB1EFBE6
:10021000F98BD89BBBAB9ABB754A545A376A167A8E
:10022000F10AD01AB32A923A2EFD0FED6CDD4DCDB6
:10023000AABD8BADE89DC98D267C076C645C454CDE
:10024000A23C832CE01CC10C1FEF3EFF5DCF7CDF86
:100250009BAFBABFD98FF89F176E367E554E745E2E
:10026000932EB23ED10EF01E0000000024002700A5
:100270002A0000000000250028002B0000000000DC
:1002800023002600290004040404040404040202D8
:100290000202020203030303030301020408102005
:1002A0004080010204081020010204081020000010
:1002B0000007000201000003040600000000000027
:1002C0000000761611241FBECFEFD8E0DEBFCDBFF1
:1002D00011E0A0E0B1E0E8EBFFE202C005900D9272
:1002E000A631B107D9F716E0A6E1B1E001C01D9231
:1002F000A03EB107E1F712E0C4ECD2E004C02297BF
:10030000FE010E94D617C23CD107C9F70E94CD1644
:100310000C94DA170C94000061E070E040E050E0CB
:1003200016C0342F2227FB01E55BFA4F8081E82FAE
:10033000F0E0852F9927E827F927EE0FFF1FE859EE
:10034000FF4F45915491422753276F5F7F4F809114
:10035000830590918405861797071CF740939D05A8
:1003600050939E05E0918305F0918405E35BFA4F7D
:100370004083E0918305F0918405E45BFA4F50835C
:1003800080918305909184050296909384058093D3
:1003900083050895AF92BF92CF92DF92EF92FF92C2
:1003A0000F931F93CF93DF931092E0041092DF041A
:1003B0008FEF8093E3041092E2041092E1048AEE3E
:1003C0008093190186EA80931A0110921B0184E040
:1003D00090E09093700480936F0483E090E090939A
:1003E00072048093710440E050E0C1E0D0E031E05D
:1003F000E32EF12C012D112D1092E2041092E10454
:10040000BE01042E02C0660F771F0A94E2F766C091
:100410008091E1049091E204FC01EE0FFF1FE80FD0
:10042000F91FE557FB4F808190E086239723892BA6
:10043000B9F0E0917104F0917204E85EFE4F208102
:1004400080916F04909170045701680104C0AA0C58
:10045000BB1CCC1CDD1C8A95D2F72A29208319C02D
:10046000E0917104F0917204E85EFE4F208180916A
:100470006F04909170045701680104C0AA0CBB1C62
:10048000CC1CDD1C8A95D2F7D601C501809582234C
:10049000808380916F049091700401969093700412
:1004A00080936F0480916F049091700408976CF0B2
:1004B0001092700410926F048091710490917204F4
:1004C000019690937204809371048091E10490915D
:1004D000E20401969093E2048093E1048091E104A8
:1004E0009091E2044C970CF493CF4F5F5F4F4830EC
:1004F000510509F081CF40E050E0C1E0D0E0B1E02B
:10050000EB2EF12C012D112D1092E2041092E1043A
:10051000BE01042E02C0660F771F0A94E2F766C080
:100520008091E1049091E204FC01EE0FFF1FE80FBF
:10053000F91FE557FB4F818190E086239723892B94
:10054000B9F0E0917104F0917204E85EFE4F2081F1
:1005500080916F04909170045701680104C0AA0C47
:10056000BB1CCC1CDD1C8A95D2F72A29208319C01C
:10057000E0917104F0917204E85EFE4F2081809159
:100580006F04909170045701680104C0AA0CBB1C51
:10059000CC1CDD1C8A95D2F7D601C501809582233B
:1005A000808380916F049091700401969093700401
:1005B00080936F0480916F049091700408976CF0A1
:1005C0001092700410926F048091710490917204E3
:1005D000019690937204809371048091E10490914C
:1005E000E20401969093E2048093E1048091E10497
:1005F0009091E2044C970CF493CF4F5F5F4F4430DF
:10060000510509F081CF44E050E0C1E0D0E031E095
:10061000E32EF12C012D112D1092E2041092E10431
:10062000BE01042E02C0660F771F0A94E2F766C06F
:100630008091E1049091E204FC01EE0FFF1FE80FAE
:10064000F91FE557FB4F818190E086239723892B83
:10065000B9F0E0917104F0917204E85EFE4F2081E0
:1006600080916F04909170045701680104C0AA0C36
:10067000BB1CCC1CDD1C8A95D2F72A29208319C00B
:10068000E0917104F0917204E85EFE4F2081809148
:100690006F04909170045701680104C0AA0CBB1C40
:1006A000CC1CDD1C8A95D2F7D601C501809582232A
:1006B000808380916F0490917004019690937004F0
:1006C00080936F0480916F049091700408976CF090
:1006D0001092700410926F048091710490917204D2
:1006E000019690937204809371048091E10490913B
:1006F000E20401969093E2048093E1048091E10486
:100700009091E2044B970CF493CF4F5F5F4F4830CA
:10071000510509F081CF40E050E0C1E0D0E0B1E008
:10072000EB2EF12C012D112D1092E2041092E10418
:10073000BE01042E02C0660F771F0A94E2F766C05E
:100740008091E1049091E204FC01EE0FFF1FE80F9D
:10075000F91FE557FB4F828190E086239723892B71
:10076000B9F0E0917104F0917204E85EFE4F2081CF
:1007700080916F04909170045701680104C0AA0C25
:10078000BB1CCC1CDD1C8A95D2F72A29208319C0FA
:10079000E0917104F0917204E85EFE4F2081809137
:1007A0006F04909170045701680104C0AA0CBB1C2F
:1007B000CC1CDD1C8A95D2F7D601C5018095822319
:1007C000808380916F0490917004019690937004DF
:1007D00080936F0480916F049091700408976CF07F
:1007E0001092700410926F048091710490917204C1
:1007F000019690937204809371048091E10490912A
:10080000E20401969093E2048093E1048091E10474
:100810009091E2044B970CF493CF4F5F5F4F4830B9
:10082000510509F081CF84E090E0909370048093AB
:100830006F0483E090E0909372048093710481E0F0
:1008400090E09093E2048093E10441E0E42EF12CE7
:10085000012D112D8EC08091E304880F8093E30455
:100860008091E3042091E30490E034E0959587952E
:100870003A95E1F781709070221F2227221F30E005
:100880008217930721F08091E304816003C0809177
:10089000E3048E7F8093E3042091E304E0917104EC
:1008A000F0917204E85EFE4F808140916F04509198
:1008B000700490E002C0959587954A95E2F730E084
:1008C0008227932780FF17C0E0917104F091720492
:1008D000E85EFE4F208180916F0490917004B80112
:1008E000A70104C0440F551F661F771F8A95D2F7D2
:1008F000242B208319C0E0917104F0917204E85E0A
:10090000FE4F208180916F0490917004570168011F
:1009100004C0AA0CBB1CCC1CDD1C8A95D2F7D601E6
:10092000C50180958223808380916F04909170042B
:1009300001969093700480936F0480916F0490915E
:10094000700408976CF01092700410926F048091FC
:1009500071049091720401969093720480937104D3
:100960008091E1049091E20401969093E2048093D7
:10097000E1048091E1049091E204855992400CF4E5
:100980006ACFDF91CF911F910F91FF90EF90DF9091
:10099000CF90BF90AF9008954091E3042091E3047D
:1009A0008091E30430E03595279550E042275327A6
:1009B0004170507090E095958795959587958170D9
:1009C00090704817590709F18091E0042091DF04E5
:1009D00090E0FC01EE0FFF1FE80FF91FE20FF11D81
:1009E000E557FB4F40812091E1043091E20481E022
:1009F00090E0A0E0B0E004C0880F991FAA1FBB1FC1
:100A00002A95D2F7482B408321C08091E0042091A1
:100A1000DF0490E0FC01EE0FFF1FE80FF91FE20F6B
:100A2000F11DE557FB4F40812091E1043091E20434
:100A300081E090E0A0E0B0E004C0880F991FAA1FF9
:100A4000BB1F2A95D2F78095842380838091E1048F
:100A50009091E20401969093E2048093E104209146
:100A6000E3048091E30490E09595879595958795AB
:100A700030E08227932780FF21C08091E0042091FD
:100A8000DF0490E0FC01EE0FFF1FE80FF91FE20FFB
:100A9000F11DE557FB4F40812091E1043091E204C4
:100AA00081E090E0A0E0B0E004C0880F991FAA1F89
:100AB000BB1F2A95D2F7482B408321C08091E004C8
:100AC0002091DF0490E0FC01EE0FFF1FE80FF91FFB
:100AD000E20FF11DE557FB4F40812091E104309179
:100AE000E20481E090E0A0E0B0E004C0880F991F2C
:100AF000AA1FBB1F2A95D2F78095842380838091FB
:100B0000E1049091E20401969093E2048093E10461
:100B10000895CF93DF931092E0041092DF041092B7
:100B2000E3041092E2041092E10481E090E045C0F9
:100B3000C0E0D0E08091E304880F8093E304E0916B
:100B40000F05F0911005EC51FB4F808190E00C2EC9
:100B500002C0959587950A94E2F780FF04C08091C2
:100B6000E304816003C08091E3048E7F8093E304FB
:100B70000E94CC048091E1049091E2040897A4F0D3
:100B80001092E2041092E1048091DF048F5F809361
:100B9000DF048091DF04833038F01092DF0480910D
:100BA000E0048F5F8093E0042196C830D10511F6F0
:100BB00080910F05909110050196909310058093F8
:100BC0000F0580910F05909110058A970CF4B0CF16
:100BD0008091E304880F8093E3048091E3048E7F87
:100BE0008093E3040E94CC048091E304880F8093F7
:100BF000E3048091E3048E7F8093E3040E94CC049D
:100C0000DF91CF9108958091E30483FFC6C0809166
:100C1000E30486FFC2C004C08091E30486FDC1C026
:100C20008091E304880F8093E3048091E3048E7F36
:100C30008093E30480917D0480FFBCC08091E30435
:100C400080FFB8C004C08091E30480FDB7C08091EC
:100C5000E0042091DF0490E0FC01EE0FFF1FE80F9D
:100C6000F91FE20FF11DE557FB4F40812091E10490
:100C70003091E20481E090E0A0E0B0E004C0880F91
:100C8000991FAA1FBB1F2A95D2F7809584238083C2
:100C90008091E0048F5F8093E0048091DF048823DB
:100CA00001F58091E0048C31E0F01092E004809135
:100CB000E1049091E20401979093E2048093E104AF
:100CC0008091E1049091E20497FF0BC087E090E0EF
:100CD0009093E2048093E1048091DF048F5F80931E
:100CE000DF048091DF04813079F48091E0048C315D
:100CF00058F01092E0048091E1049091E204019791
:100D00009093E2048093E1048091DF048130A9F4A0
:100D10008091E0048B3189F48091E1049091E204A8
:100D200004975CF41092E0048091E1049091E20455
:100D300001979093E2048093E1048091E104909103
:100D4000E20497FF0BC087E090E09093E204809369
:100D5000E1048091DF048F5F8093DF048091DF04E2
:100D6000823009F04CC08091E0048B3108F447C018
:100D70001092E0048091E1049091E2040197909335
:100D8000E2048093E1048091E1049091E20497FFF2
:100D900036C083E08093880508958091E30483FF43
:100DA0003BCF8091E304880F8093E3048091E304B8
:100DB00081603ECF80917D0480FF45CF8091E0042B
:100DC0002091DF0490E0FC01EE0FFF1FE80FF91FF8
:100DD000E20FF11DE557FB4F40812091E104309176
:100DE000E20481E090E0A0E0B0E004C0880F991F29
:100DF000AA1FBB1F2A95D2F7482B408349CF0895DD
:100E00008091E30487FF19C08091E30482FF15C03D
:100E100004C08091E30482FD14C08091E3048E7FBE
:100E20008093E30480910E0590E0959587958093DB
:100E30000E0580910E058F7713C08091E30487FF24
:100E4000E8CF8091E30481608093E30480910E05F4
:100E500090E09595879580930E0580910E058068AA
:100E600080930E058091E304880F8093E304089536
:100E700080918A048F5F80938A0480918A048830ED
:100E800000F110928A04E0910201F0910301E85E02
:100E9000FE4F808180937304809102019091030141
:100EA0000197909303018093020180910201909138
:100EB0000301892B31F48CE291E09093030180933C
:100EC0000201E6E1F0E0DF01AD58BB4F8C9190E00C
:100ED000959587958C939F0121503040F901ED58ED
:100EE000FB4F808180FF03C08C91806802C08C9191
:100EF0008F778C938FEF2F3F380711F0F901E3CFF5
:100F0000089580919F059091A00501969093A0056A
:100F100080939F0580918E05882331F485E00E949F
:100F20006114892B51F005C085E00E946114892B62
:100F300021F480911601806803C0809116018F779B
:100F400080931601809117018F5F80931701809124
:100F50001701883009F5E0910001F09101018091BD
:100F60001601E85EFE4F808380910001909101019F
:100F7000019790930101809300018091000190916D
:100F80000101892B31F48CE291E09093010180936F
:100F900000011092170107C08091160190E095950D
:100FA00087958093160181E080938A05089580914A
:100FB0009F059091A00501969093A00580939F05B1
:100FC0008091940590919505019790939505809354
:100FD000940580918B05843021F080918B058530BC
:100FE00059F510929B0510929A0580919C058150AD
:100FF00080939C0586E00E946114019719F486E0B5
:1010000060E002C086E061E00E940D1480918B05D3
:10101000853091F480918F05882331F486E00E9419
:101020006114019749F405C086E00E946114892B80
:1010300019F486E080938B0580918B05873029F029
:1010400080918B05883009F079C080919A05909144
:101050009B05019690939B0580939A0580919A0534
:1010600090919B05803691055CF010929B05109243
:101070009A05809199058F5F8093990580919905D4
:10108000E0916D04F0916E04E85EFE4F8081209146
:101090006F043091700490E002C0959587952A9571
:1010A000E2F780FF05C080918F05813029F407C0E9
:1010B00080918F05813019F486E061E002C086E0FE
:1010C00060E00E940D1480916F049091700401966D
:1010D0009093700480936F0480916F0490917004DA
:1010E0000897D1F41092700410926F0480916D04EF
:1010F00090916E04019690936E0480936D0480919C
:101100006D0490916E048355934034F081E090E03B
:1011100090936E0480936D0480918B05883071F4F8
:1011200020916B0430916C0480916D0490916E0459
:101130002817390719F489E080938B0581E08093A3
:101140008D0583E160E00E940D1408958091810473
:101150008A3AC1F4809180048A3AA1F480917F0494
:101160008A3A81F480917E048A3A61F481E0809326
:1011700088058091970581608093970589E060E0FC
:101180000E940D1408958FE190E029C08091A1057F
:101190009091A205A091A305B091A4052091A50569
:1011A0003091A60504C0B595A795979587952A9582
:1011B000D2F780FF03C08AE061E002C08AE060E00D
:1011C0000E940D1487E061E00E940D1487E060E04A
:1011D0000E940D148091A5059091A605019790930A
:1011E000A6058093A5058091A5059091A60597FF7A
:1011F000CDCF8CE061E00E940D148CE060E00E9495
:101200000D148AE060E00E940D14089585E591E3D5
:10121000A0E0B0E08093A1059093A205A093A30560
:10122000B093A4050E94C30882E990EDA5E1B1E066
:101230008093A1059093A205A093A305B093A40564
:101240000E94C30883EA90E0A5E1BBE28093A10578
:101250009093A205A093A305B093A4050E94C30890
:1012600084E190EBA7E3B0E08093A1059093A20501
:10127000A093A305B093A4050E94C30880E890E45E
:10128000A1E6B9E18093A1059093A205A093A305DF
:10129000B093A4050E94C308089582E990EDA5E7E4
:1012A000B0E08093A1059093A205A093A305B0930D
:1012B000A4050E94C30883E291E8A4E1BBE2809305
:1012C000A1059093A205A093A305B093A4050E9445
:1012D000C30884E198E3A9E5B0E08093A105909369
:1012E000A205A093A305B093A4050E94C30880E5BE
:1012F00095E5A1E6B1E18093A1059093A205A093A5
:10130000A305B093A4050E94C308089581E190E568
:10131000A7E5B0E08093A1059093A205A093A30553
:10132000B093A4050E94C30883EA90E0A5E1B8E267
:101330008093A1059093A205A093A305B093A40563
:101340000E94C30880E890E4A1E6B9E18093A1057A
:101350009093A205A093A305B093A4050E94C3088F
:1013600085E591E3A0E0B0E08093A1059093A2050C
:10137000A093A305B093A4050E94C30884E190EB59
:10138000A7E3B0E08093A1059093A205A093A305E5
:10139000B093A4050E94C30882E990EDA5E1B1E0F5
:1013A0008093A1059093A205A093A305B093A405F3
:1013B0000E94C3088FE090E0AEE0B0E08093A1050A
:1013C0009093A205A093A305B093A4050E94C3081F
:1013D00086EC92E7A9E0B5E08093A1059093A20581
:1013E000A093A305B093A4050E94C30889EE91E3DE
:1013F000A2E0B0E08093A1059093A205A093A3057D
:10140000B093A4050E94C3088AE595E3A6E9B2E378
:101410008093A1059093A205A093A305B093A40582
:101420000E94C3088BE390E0A0E0B0E08093A105A8
:101430009093A205A093A305B093A4050E94C308AE
:101440008CE091E0A0E0B0E08093A1059093A2052C
:10145000A093A305B093A4050E94C3088DE090E07B
:10146000A0E0B0E08093A1059093A205A093A3050E
:10147000B093A4050E94C3080895CF93DF9380ED35
:1014800080934C050E948C01C1E0D0E009C0FE01B0
:10149000E55BFA4F608185EB96E00E943616219657
:1014A00080918305909184058C179D0784F7DF91C7
:1014B000CF910895FF920F931F93809181048A3AF0
:1014C00009F050C0809180048A3A09F04BC08091A5
:1014D0007F048E3609F046C080917E048A3009F080
:1014E00041C082E0809388051092DF041092E004EE
:1014F00087E090E09093E2048093E1048FEF809383
:10150000E30410928705809104018F5F80930401AA
:10151000F3E0FF2EF0924D0510924E0585E1809389
:101520004F05109250051092510506E010E01093FF
:101530008405009383050E943D0AF0924D051092A8
:101540004E0586E180934F058091040180935005FC
:10155000809187058093510510938405009383053E
:101560000E943D0A1F910F91FF9008951092E00490
:101570001092DF041092E3041092100510920F05F0
:1015800014C110920E058091E00490E02091DF04D8
:10159000FC01EE0FFF1FE80FF91FE20FF11DE557E9
:1015A000FB4F808186FF04C08091E304806803C004
:1015B0008091E3048F778093E3040E940007809179
:1015C000E00490E02091DF04FC01EE0FFF1FE80F24
:1015D000F91FE20FF11DE557FB4F808184FF04C026
:1015E0008091E304806803C08091E3048F77809347
:1015F000E3040E9400078091E00490E02091DF0462
:10160000FC01EE0FFF1FE80FF91FE20FF11DE55778
:10161000FB4F808182FF04C08091E304806803C097
:101620008091E3048F778093E3040E940007809108
:10163000E00490E02091DF04FC01EE0FFF1FE80FB3
:10164000F91FE20FF11DE557FB4F808180FF04C0B9
:101650008091E304806803C08091E3048F778093D6
:10166000E3040E9400078091DF048F5F8093DF0412
:101670008091DF04833038F01092DF048091E00421
:101680008F5F8093E0048091E00490E02091DF047C
:10169000FC01EE0FFF1FE80FF91FE20FF11DE557E8
:1016A000FB4F808186FF04C08091E304806803C003
:1016B0008091E3048F778093E3040E940007809178
:1016C000E00490E02091DF04FC01EE0FFF1FE80F23
:1016D000F91FE20FF11DE557FB4F808184FF04C025
:1016E0008091E304806803C08091E3048F77809346
:1016F000E3040E9400078091E00490E02091DF0461
:10170000FC01EE0FFF1FE80FF91FE20FF11DE55777
:10171000FB4F808182FF04C08091E304806803C096
:101720008091E3048F778093E3040E940007809107
:10173000E00490E02091DF04FC01EE0FFF1FE80FB2
:10174000F91FE20FF11DE557FB4F808180FF04C0B8
:101750008091E304806803C08091E3048F778093D5
:10176000E3040E9400078091DF048F5F8093DF0411
:101770008091DF04833038F01092DF048091E00420
:101780008F5F8093E004E0910F05F0911005809148
:101790000E05EC51FB4F808380910F059091100551
:1017A00001969093100580930F0580910F059091FD
:1017B000100589970CF4E5CE84E0809388058FE2CC
:1017C00080934D0510924E0587E180934F058091DF
:1017D00004018093500580918705809351051092F4
:1017E0005205109253051092100510920F0517C064
:1017F000A0910F05B0911005E0910F05F091100533
:10180000EC51FB4F8081AC5ABA4F8C9380910F05FD
:101810009091100501969093100580930F0580918B
:101820000F059091100589971CF382E390E0909347
:101830008405809383050E943D0A089590911405C4
:10184000913109F042C090934D0510924E0581E907
:1018500080934F0582E2809350059093510584E474
:101860008093520586E5809353058DE2809354055D
:101870008DE48093550585E48093560587E4809335
:10188000570581E48093580580E28093590582E5ED
:1018900080935A0591E390935B058EE280935C05FB
:1018A00090935D0582E380935E0582E480935F05FB
:1018B00084E190E090938405809383050E943D0A23
:1018C00081E080938B058093890580911405823196
:1018D000E1F485E080934D0510924E0582E98093F6
:1018E0004F0583E18093500589E08093510580E1A5
:1018F0008093520581E08093530588E090E09093B7
:101900008405809383050E943D0A809114058431EB
:1019100009F054C080911505803CE9F580911705C8
:101920008093900580911805809391058091190509
:101930008093920580911A0580939305809190057C
:1019400080FF04C081E080938E0502C010928E0556
:101950008091900581FF04C081E080938F0502C0D3
:1019600010928F058091900582FF03C01092A70509
:1019700003C081E08093A7058091900582FF03C09A
:101980001092A80503C081E08093A80581E08093B0
:10199000A7058093A80582E080934D0510924E051F
:1019A00084E980934F0586E08093500585E090E0C0
:1019B00090938405809383050E943D0A80911405CD
:1019C0008031D1F4909112059230B1F480911505D7
:1019D0008093960590934D0510924E0580E9809373
:1019E0004F0586E08093500585E090E09093840554
:1019F000809383050E943D0A80911405803169F52A
:101A000080911205813049F588E080934D05109250
:101A10004E0580E980934F0587E4809350058091BF
:101A2000970580935105809189058093520585E142
:101A3000809353058CEF8093540580919805809393
:101A4000550580919905809356058BE090E0909321
:101A50008405809383050E943D0A80911405863198
:101A600071F480918F05813019F486E061E002C045
:101A700086E060E00E940D1481E080938C058091E7
:101A80001405873151F580911505809304018091EB
:101A900016058093870521E030E0F901E85EFA4FF2
:101AA0008081F901EC51FB4F80832F5F3F4F2A3239
:101AB000310599F786E590E090936C0480936B0470
:101AC00081E090E090936E0480936D040E948905FC
:101AD0000E94CA0182E080938C05809114058931AF
:101AE00009F03EC01092A00510929F0580918605D6
:101AF0008F5F8093860580918605853110F0109266
:101B0000860528E030E041E050E0E0916B04F09180
:101B10006C04D901AF5EBA4F8C91E85EFE4F8083B2
:101B200080916B0490916C04019690936C04809367
:101B30006B0480916B0490916C048355934024F066
:101B400050936C0440936B042F5F3F4F2431310559
:101B5000E1F680918C05823019F483E080938C0546
:101B6000809114058A3109F04DC180916B049091E8
:101B70006C04019790936C0480936B0480916B04C8
:101B800090916C04892B31F482E593E090936C047E
:101B900080936B0480916B0490916C0401979093F7
:101BA0006C0480936B0480916B0490916C04892B7E
:101BB00031F482E593E090936C0480936B04809100
:101BC0006B0490916C04019790936C0480936B0468
:101BD00080916B0490916C04892B31F482E593E041
:101BE00090936C0480936B04E0916B04F0916C040F
:101BF000E85EFE4F85E5808380916B0490916C04D4
:101C0000019690936C0480936B0480916B04909187
:101C10006C048355934034F081E090E090936C0421
:101C200080936B04E0916B04F0916C04E85EFE4FCE
:101C300085E5808380916B0490916C04019690936C
:101C40006C0480936B0480916B0490916C048355B9
:101C5000934034F081E090E090936C0480936B04A7
:101C6000E0916B04F0916C04E85EFE4F85E58083A3
:101C700080916B0490916C04019690936C04809316
:101C80006B0480916B0490916C048355934034F005
:101C900081E090E090936C0480936B04E0916B047E
:101CA000F0916C04E85EFE4F85E5808380916B04C3
:101CB00090916C04019690936C0480936B048091D6
:101CC0006B0490916C048355934034F081E090E074
:101CD00090936C0480936B04E0916B04F0916C041E
:101CE000E85EFE4F88EC808380916B0490916C04D9
:101CF000019690936C0480936B0480916B04909197
:101D00006C048355934034F081E090E090936C0430
:101D100080936B04E0916B04F0916C04E85EFE4FDD
:101D20008AE7808380916B0490916C040196909374
:101D30006C0480936B0480916B0490916C048355C8
:101D4000934034F081E090E090936C0480936B04B6
:101D5000E0916B04F0916C04E85EFE4F108280917C
:101D60006B0490916C04019690936C0480936B04C7
:101D700080916B0490916C048355934034F081E022
:101D800090E090936C0480936B04E0916B04F0916D
:101D90006C04E85EFE4F108280916B0490916C049D
:101DA000019690936C0480936B0480916B049091E6
:101DB0006C048355934034F081E090E090936C0480
:101DC00080936B04E0916B04F0916C04E85EFE4F2D
:101DD000108280916B0490916C04019690936C0436
:101DE00080936B0480916B0490916C0483559340B5
:101DF00034F081E090E090936C0480936B0484E075
:101E000080938C05809114058F31E1F59091150533
:101E1000903CD1F486E080934D0510924E058FE9F9
:101E200080934F05909350051092510510925205E2
:101E3000109253051092540589E090E09093840528
:101E4000809383050E943D0A90911505913CD1F441
:101E500086E080934D0510924E058FE980934F05E3
:101E6000909350051092510510925205109253050F
:101E70001092540589E090E0909384058093830547
:101E80000E943D0A109211051092120510924A0507
:101E900010924905089583E180934D0510924E05F7
:101EA00089E180934F0580910401809350058091D2
:101EB00087058093510588EE8093520583E08093D7
:101EC000530525E130E04EE150E0FA01E21BF30B4F
:101ED000D901AD58BB4F8C91E55BFA4F80832150FF
:101EE00030402930310589F7109260051092610564
:101EF00086E190E090938405809383050E943D0ADB
:101F0000089583E080934D0510924E058AE18093F9
:101F10004F0580910401809350058091870580933F
:101F2000510586E090E090938405809383050E949C
:101F30003D0A08958091A8050E94611380E061E840
:101F400077E043E050E00E943E13809197058E7F3A
:101F500080939705809197058D7F8093970588E002
:101F600060E00E940D148091A705882311F40E945F
:101F700006098CE291E09093010180930001109298
:101F80008A041092880589E061E00E940D14109285
:101F9000850510928605109299051092980581E0AA
:101FA00080938B0510928C058093890508950F937B
:101FB0001F93CF93DF9385EB96E00E94C915181607
:101FC00019060CF50091490510914A0585EB96E03C
:101FD0000E94FD150F5E1A4FF8018083809149051C
:101FE00090914A05019690934A0580934905809106
:101FF000490590914A05C89734F087E390E09093A3
:102000004A058093490580911105803D21F0109289
:102010004A051092490580911105803D99F48091FF
:10202000490590914A0505976CF02091490530913A
:102030004A058091120590E004968217930714F4E4
:102040000E941E0C80918D05813009F045C02091C1
:102050006B0430916C0480916D0490916E04821732
:10206000930784F480916B0490916C0420916D042B
:1020700030916E04821B930B6CE070E00E948B1712
:102080006093980520916B0430916C0480916D04ED
:1020900090916E042817390794F480916B04909105
:1020A0006C0420916D0430916E048E5A9C4F821BFB
:1020B000930B6CE070E00E948B1760939805209161
:1020C0006B0430916C0480916D0490916E0428171C
:1020D000390711F41092980580918B05882309F433
:1020E000EAC080918B05813009F056C080918C0543
:1020F000882309F451C08AEF90E090930301809304
:1021000002018CE291E0909301018093000180E054
:102110000E946113809197058E7F8093970580912F
:10212000970582608093970588E061E00E940D1416
:102130008091A705882311F40E944D098091A8057C
:1021400067ED77E042E050E00E943E1380919205F7
:1021500025E0829FC00111249093950580939405FA
:1021600040919405509195058091930590E02BEF57
:1021700034E0BC01629FC001639F900D729F900D7F
:102180001124840F951F909395058093940582E008
:1021900080938B058093890580918B05823049F46B
:1021A0008091940590919505059718F483E08093AC
:1021B0008B0590918B05933061F480918C05823072
:1021C00040F080E480939C0584E080938B0590939D
:1021D000890580918B05843039F480919C0582308B
:1021E00018F485E080938B0580918B05863031F45F
:1021F00087E080938B0585E08093890580918B052E
:10220000873009F045C080919F059091A005815CC1
:10221000924110F00E949A0F809198058530D0F479
:1022200080916D0490916E04CC9790936E0480938E
:102230006D0480916D0490916E041816190654F087
:1022400080916D0490916E048E5A9C4F90936E0411
:1022500080936D04809198058334D0F080916B0455
:1022600090916C04CC9790936C0480936B04809154
:102270006B0490916C041816190654F080916B044D
:1022800090916C048E5A9C4F90936C0480936B04D5
:1022900090918B05973049F480918C05843029F416
:1022A00088E080938B059093890580918B05893018
:1022B00011F40E949A0F809188058630C0F5209114
:1022C0000001309101018091020190910301821778
:1022D000930794F4809102019091030120910001F1
:1022E00030910101845D9E4F821B930B8B3F9105C2
:1022F0001CF081E080938A05209102013091030156
:1023000080910001909101018217930784F48091DC
:102310000201909103012091000130910101821B83
:10232000930B8B3F91051CF081E080938A0580918F
:102330008A05813009F035C10E94380780918805EF
:10234000882331F480918A05813011F40E94A60817
:1023500080918805813031F480918A05813011F4B3
:102360000E945A0A80918805823061F480918A0522
:10237000813041F40E94030610928B0583E161E0F5
:102380000E940D1480918805833031F480918A0574
:10239000813011F40E94B60A80918805843039F4A6
:1023A00080918A05813019F485E0809388058091B9
:1023B00088058530D1F480918A058130B1F405C05B
:1023C0000E943807809185058F5F809385058091F5
:1023D00085058131A8F386E08093880510928505F4
:1023E00085E18093860510928A0580918805863064
:1023F00009F0D7C080918A05813009F0D2C0809160
:1024000085058F5F8093850580918505823008F46E
:102410004FC080918505893108F04AC020910201A2
:10242000309103018091000190910101821793077F
:10243000CCF4809102019091030120910001309130
:102440000101821B930B45976CF0C1E0D0E00E9424
:102450003807809185058F5F809385052196C1326D
:10246000D105A9F72091020130910301809100016B
:102470009091010128173907DCF4809102019091B5
:1024800003012091000130910101845D9E4F821B68
:10249000930B45976CF0C1E0D0E00E943807809123
:1024A00085058F5F809385052196C132D105A9F7F7
:1024B000809185058934E1F480917F048535C1F4EC
:1024C00080917E048535A1F480917D04853581F469
:1024D00080917C04853561F480917B04883C41F4D3
:1024E00080917A048A3721F40E949A0F0E94810F0A
:1024F000809186058431A1F480918505823480F035
:1025000080917E04853561F480917D048D3241F4A3
:1025100080917C04863121F410928A050E9438074C
:1025200080918605843111F5809185058934F1F417
:1025300080917F048535F1F580917E048D32D1F54F
:1025400080917D048631B1F511C080917E048D3279
:1025500021F080917D04863191F585E580937F049B
:102560008DE280937E0486E180937D0480918505D1
:10257000893431F480918605809387050E944B0F42
:1025800080918505803668F01092850580918605DA
:102590008F5F8093860580918605853110F01092BB
:1025A000860510928A0510928D05DF91CF911F91BB
:1025B0000F91089580917F04853539F6CECF0E9422
:1025C0009A0F0E94810FD2CF0F931F938DE061E08D
:1025D0000E94CE1383E161E00E94CE1385E060E0AB
:1025E0000E94CE1382E060E00E94CE1383E060E0A0
:1025F0000E94CE1386E061E00E94CE1387E061E086
:102600000E94CE1388E061E00E94CE1389E061E071
:102610000E94CE138CE061E00E94CE138AE061E05C
:102620000E94CE1388E060E00E940D1489E061E012
:102630000E940D1487E060E00E940D148CE060E0C1
:102640000E940D148AE060E00E940D1405EB16E074
:10265000C80140E052EC61E070E00E944215C80100
:102660000E94261680E061E877E043E050E00E9497
:102670003E130E9486091F910F910895823000F544
:10268000E82FF0E0EE0FFF1FE755FA4F71836083EC
:10269000882319F08130A1F408C0809169008C7FF3
:1026A000842B80936900E89A089580916900440F13
:1026B000551F440F551F837F842B80936900E99A2F
:1026C0000895823080F4882319F0813021F402C00B
:1026D000E89801C0E998E82FF0E0EE0FFF1FE755FA
:1026E000FA4F1182108208951F920F920FB60F9227
:1026F00011242F933F934F935F936F937F938F9307
:102700009F93AF93BF93EF93FF938091A90590910F
:10271000AA05892B29F0E091A905F091AA05099550
:10272000FF91EF91BF91AF919F918F917F916F91A9
:102730005F914F913F912F910F900FBE0F901F907F
:1027400018951F920F920FB60F9211242F933F935B
:102750004F935F936F937F938F939F93AF93BF93A9
:10276000EF93FF938091AB059091AC05892B29F0F5
:10277000E091AB05F091AC050995FF91EF91BF9108
:10278000AF919F918F917F916F915F914F913F9109
:102790002F910F900FBE0F901F901895CF93DF933E
:1027A000482F50E0CA0186569D4FFC0134914A578C
:1027B0005D4FFA018491882369F190E0880F991F99
:1027C000FC01E859FD4FA591B491FC01EE58FD4F75
:1027D000C591D491662351F42FB7F8948C91932F1F
:1027E000909589238C93888189230BC0623061F492
:1027F0002FB7F8948C91932F909589238C9388818F
:10280000832B88832FBF06C09FB7F8948C91832BAE
:102810008C939FBFDF91CF910895482F50E0CA015C
:1028200082559D4FFC012491CA0186569D4FFC01A3
:1028300094914A575D4FFA013491332309F440C013
:10284000222351F1233071F0243028F42130A1F0FB
:10285000223011F514C02630B1F02730C1F02430F9
:10286000D9F404C0809180008F7703C080918000EC
:102870008F7D8093800010C084B58F7702C084B5AF
:102880008F7D84BD09C08091B0008F7703C0809197
:10289000B0008F7D8093B000E32FF0E0EE0FFF1FBC
:1028A000EE58FD4FA591B4912FB7F894662321F40B
:1028B0008C919095892302C08C91892B8C932FBF8A
:1028C0000895682F70E0CB0182559D4FFC01249143
:1028D000CB0186569D4FFC0144916A577D4FFB0109
:1028E0009491992319F420E030E03CC0222351F167
:1028F000233071F0243028F42130A1F0223011F57A
:1029000014C02630B1F02730C1F02430D9F404C00F
:10291000809180008F7703C0809180008F7D8093AD
:10292000800010C084B58F7702C084B58F7D84BDD0
:1029300009C08091B0008F7703C08091B0008F7D77
:102940008093B000892F90E0880F991F84589D4F85
:10295000FC01A591B4918C9120E030E0842311F02A
:1029600021E030E0C901089508951F920F920FB63B
:102970000F9211242F933F934F938F939F93EF9335
:10298000FF938091C00082FD1DC04091C600209140
:102990002D0630912E062F5F3F4F2F77307080919C
:1029A0002F06909130062817390771F0E0912D0617
:1029B000F0912E06E355FA4F408330932E06209374
:1029C0002D0602C08091C600FF91EF919F918F91DB
:1029D0004F913F912F910F900FBE0F901F90189520
:1029E000E091C106F091C206E058FF4F81919191AC
:1029F0002081318180589F4F821B930B60E870E0EB
:102A00000E948B17892B11F00E94B41408951F9215
:102A10000F920FB60F9211242F933F938F939F9392
:102A2000EF93FF932091B1063091B2068091B306E7
:102A30009091B4062817390731F48091C1008F7D39
:102A40008093C10014C0E091B306F091B406EF5C2E
:102A5000F94F20818091B3069091B40601968F774B
:102A600090709093B4068093B3062093C600FF91B4
:102A7000EF919F918F913F912F910F900FBE0F90EB
:102A80001F901895AF92BF92DF92EF92FF920F9333
:102A90001F93CF93DF93EC017A018B01DD2440304B
:102AA00081EE580780E0680780E0780711F0DD24A8
:102AB000D39491E0A92EB12CEC89FD89DD2069F039
:102AC000C50108A002C0880F991F0A94E2F780830D
:102AD00060E079E08DE390E005C0108260E874E882
:102AE0008EE190E0A80197010E949E17215030408E
:102AF00040405040569547953795279580E12030C6
:102B0000380720F0DD2011F0DD24D6CFE889F989DF
:102B10003083EA89FB89208319A2EE89FF894081ED
:102B200021E030E0C9010C8C02C0880F991F0A9483
:102B3000E2F7482B4083EE89FF894081C9010D8C63
:102B400002C0880F991F0A94E2F7482B4083EE8950
:102B5000FF894081C9010E8C02C0880F991F0A9419
:102B6000E2F7482B4083EE89FF8980810F8C02C0F9
:102B7000220F331F0A94E2F7209528232083DF9148
:102B8000CF911F910F91FF90EF90DF90BF90AF908A
:102B90000895DC011C96ED91FC911D97E058FF4FC4
:102BA000819191912081318180589F4F821B930B9D
:102BB00060E870E00E948B170895DC011C96ED918F
:102BC000FC911D97E058FF4F20813181E058F04083
:102BD000DF01AE57BF4F8D919C9111972817390790
:102BE00019F42FEF3FEF07C08D919C91E80FF91F6B
:102BF0008081282F30E0C9010895DC011C96ED91F9
:102C0000FC911D97E058FF4F20813181E058F04042
:102C1000DF01AE57BF4F8D919C911197281739074F
:102C200019F42FEF3FEF10C08D919C911197E80F91
:102C3000F91F20818D919C91119701968F7790704B
:102C400011969C938E9330E0C9010895DC01919612
:102C50008C919197882339F05496ED91FC9155977A
:102C6000808186FFF9CF91961C920895CF93DF93D0
:102C7000EC01EE85FF85E058FF4F20813181E0585F
:102C8000F0402F5F3F4F2F773070DF01AE57BF4FBF
:102C90008D919C91119728173907D1F3E058FF4F78
:102CA00080819181E058F040E80FF91F6083EE8544
:102CB000FF85E058FF4F31832083EE89FF89208113
:102CC00081E090E00F8C02C0880F991F0A94E2F710
:102CD000282B208381E089A3EC89FD898081806491
:102CE000808381E090E0DF91CF9108951092B80643
:102CF0001092B70688EE93E0A0E0B0E08093B906AA
:102D00009093BA06A093BB06B093BC0689E091E00D
:102D10009093B6068093B5068DEA95E09093C2062F
:102D20008093C10681E396E09093C4068093C30626
:102D300085EC90E09093C6068093C50684EC90E005
:102D40009093C8068093C70680EC90E09093CA06E3
:102D50008093C90681EC90E09093CC068093CB06DB
:102D600082EC90E09093CE068093CD0686EC90E0C6
:102D70009093D0068093CF0684E08093D10683E0C1
:102D80008093D20687E08093D30685E08093D406B3
:102D900081E08093D50608950895CF93DF930E9434
:102DA00050170E94CC160E94E412C0EFD4E10E949A
:102DB000D70F2097E1F30E94F014F9CFCF92DF9262
:102DC000EF92FF920F931F93CF93DF937C016B01E0
:102DD0008A01C0E0D0E00FC0D6016D916D01D7012E
:102DE000ED91FC910190F081E02DC7010995C80F8C
:102DF000D91F015010400115110571F7CE01DF9167
:102E0000CF911F910F91FF90EF90DF90CF90089599
:102E10001F920F920FB60F9211242F933F938F930F
:102E20009F93AF93BF938091DB069091DC06A091B6
:102E3000DD06B091DE063091DF060196A11DB11DC1
:102E4000232F2D5F2D3720F02D570196A11DB11D89
:102E50002093DF068093DB069093DC06A093DD06CB
:102E6000B093DE068091D7069091D806A091D9063E
:102E7000B091DA060196A11DB11D8093D7069093FB
:102E8000D806A093D906B093DA06BF91AF919F916F
:102E90008F913F912F910F900FBE0F901F9018951B
:102EA000789484B5826084BD84B5816084BD85B525
:102EB000826085BD85B5816085BDEEE6F0E08081EC
:102EC00081608083E1E8F0E010828081826080830D
:102ED000808181608083E0E8F0E080818160808390
:102EE000E1EBF0E0808184608083E0EBF0E08081C2
:102EF00081608083EAE7F0E0808184608083808164
:102F0000826080838081816080838081806880830B
:102F10001092C100089597FB092E07260AD077FD6D
:102F200004D02ED006D000201AF4709561957F4F02
:102F30000895F6F7909581959F4F0895A1E21A2E76
:102F4000AA1BBB1BFD010DC0AA1FBB1FEE1FFF1F4D
:102F5000A217B307E407F50720F0A21BB30BE40B9D
:102F6000F50B661F771F881F991F1A9469F76095E4
:102F70007095809590959B01AC01BD01CF0108959E
:102F8000AA1BBB1B51E107C0AA1FBB1FA617B7078F
:102F900010F0A61BB70B881F991F5A95A9F78095AB
:102FA0009095BC01CD010895EE0FFF1F0590F4919F
:082FB000E02D0994F894FFCF15
:102FB8002C01FA0001000000003616DE16C915FDC6
:062FC80015DD15261600C0
:00000001FF
